:100000000C9462000C948A000C948A000C948A0070
:100010000C948A000C948A000C948A000C948A0038
:100020000C948A000C948A000C948A000C948A0028
:100030000C948A000C948A000C948A000C948A0018
:100040000C9446020C948A000C94B6020C94900214
:100050000C948A000C948A000C948A000C948A00F8
:100060000C948A000C948A000000000025002800EF
:100070002B0000000000240027002A0000000000E0
:1000800023002600290004040404040404040202DA
:100090000202020203030303030301020408102007
:1000A0004080010204081020010204081020000012
:1000B0000008000201000003040700000000000027
:1000C0000000E80211241FBECFEFD8E0DEBFCDBF95
:1000D00011E0A0E0B1E0E6E5F5E102C005900D9287
:1000E000A833B107D9F721E0A8E3B1E001C01D9220
:1000F000A33FB207E1F710E0C2E6D0E004C02197C9
:10010000FE010E94A30AC136D107C9F70E942D0340
:100110000C94A90A0C940000833081F028F48130FB
:1001200099F08230A9F008958730A9F08830C9F09D
:100130008430B1F4809180008F7D03C08091800075
:100140008F7780938000089584B58F7784BD08955C
:1001500084B58F7DFBCF8091B0008F778093B00006
:1001600008958091B0008F7DF9CFCF93DF93282F32
:1001700030E0F901E255FF4F8491F901E656FF4F57
:10018000D491F901EA57FF4FC491CC23A1F081111A
:100190000E948C00EC2FF0E0EE0FFF1FE458FF4FA1
:1001A000A591B491EC91ED2381E090E009F480E019
:1001B000DF91CF91089580E090E0FACFCF93DF9365
:1001C00090E0FC01E656FF4F24918A579F4FFC01B7
:1001D00084918823C9F090E0880F991FFC01EE58A4
:1001E000FF4FA591B491FC01E859FF4FC591D491FF
:1001F00061110DC09FB7F8948C91209582238C9348
:100200008881282328839FBFDF91CF910895623092
:1002100051F49FB7F8943C91822F809583238C935F
:10022000E8812E2BEFCF8FB7F894EC912E2B2C93E7
:100230008FBFEACF8E50806480937C0080917A00DB
:10024000806480937A0080917A0086FDFCCF809153
:100250007800909179000895AF92BF92CF92DF928B
:10026000EF92FF920F931F93CF93DF936C017B016B
:100270008B01040F151FEB015E01AE18BF08C017FC
:10028000D10759F06991D601ED91FC910190F0816F
:10029000E02DC6010995892B79F7C501DF91CF9132
:1002A0001F910F91FF90EF90DF90CF90BF90AF9094
:1002B0000895FC01538D448D252F30E0842F90E06C
:1002C000821B930B541710F0CF9608950197089551
:1002D000FC01918D828D981761F0A28DAE0FBF2F1A
:1002E000B11D5D968C91928D9F5F9F73928F90E070
:1002F00008958FEF9FEF0895FC01918D828D9817DF
:1003000031F0828DE80FF11D858D90E008958FEF1B
:100310009FEF0895FC01918D228D892F90E0805CE4
:100320009F4F821B91098F739927089587E491E06D
:100330000E948A0121E0892B09F420E0822F089590
:1003400080E090E0892B29F00E94960181110C94A5
:1003500000000895FC01A48DA80FB92FB11DA35A68
:10036000BF4F2C91848D90E001968F739927848FD5
:10037000A689B7892C93A089B1898C9183708064F8
:100380008C93938D848D981306C00288F389E02D99
:1003900080818F7D80830895EF92FF920F931F934A
:1003A000CF93DF93EC0181E0888F9B8D8C8D981328
:1003B0001AC0E889F989808185FF15C09FB7F89434
:1003C000EE89FF896083E889F98980818370806480
:1003D00080839FBF81E090E0DF91CF911F910F91CB
:1003E000FF90EF900895F62E0B8D10E00F5F1F4FDA
:1003F0000F731127E02E8C8D8E110CC00FB607FCE9
:10040000FACFE889F989808185FFF5CFCE010E9476
:10041000AA01F1CFEB8DEC0FFD2FF11DE35AFF4F39
:10042000F0829FB7F8940B8FEA89FB898081806204
:10043000CFCFCF93DF93EC01888D8823B9F0AA89C1
:10044000BB89E889F9898C9185FD03C0808186FD8F
:100450000DC00FB607FCF7CF8C9185FFF2CF8081DE
:1004600085FFEDCFCE010E94AA01E9CFDF91CF91A8
:100470000895FC0101900020E9F73197AF01481B76
:10048000590BBC0187E491E00C942C011F920F9250
:100490000FB60F9211242F933F938F939F93AF9397
:1004A000BF938091430190914401A0914501B09187
:1004B00046013091420123E0230F2D3758F5019674
:1004C000A11DB11D209342018093430190934401EB
:1004D000A0934501B093460180913E0190913F0168
:1004E000A0914001B09141010196A11DB11D8093E1
:1004F0003E0190933F01A0934001B0934101BF9111
:10050000AF919F918F913F912F910F900FBE0F90C0
:100510001F90189526E8230F0296A11DB11DD2CF7A
:100520001F920F920FB60F9211242F933F934F9368
:100530005F936F937F938F939F93AF93BF93EF934B
:10054000FF9387E491E00E94AA01FF91EF91BF9190
:10055000AF919F918F917F916F915F914F913F915B
:100560002F910F900FBE0F901F9018951F920F9212
:100570000FB60F9211242F938F939F93EF93FF93B6
:10058000E0915701F09158018081E0915D01F09177
:100590005E0182FD1BC09081809160018F5F8F732F
:1005A00020916101821741F0E0916001F0E0E95B88
:1005B000FE4F958F80936001FF91EF919F918F91F6
:1005C0002F910F900FBE0F901F9018958081F4CF40
:1005D000E7E4F1E01382128288EE93E0A0E0B0E05D
:1005E00084839583A683B78384E191E0918380839C
:1005F00085EC90E09587848784EC90E097878687E8
:1006000080EC90E0918B808B81EC90E0938B828BDF
:1006100082EC90E0958B848B86EC90E0978B868BB8
:10062000118E128E138E148EE7EEF1E082E390E0CD
:10063000A0E0B0E080839183A283B383148215820B
:100640001682178281E08087818712861386E4EE06
:10065000F1E01082118212820895CF93DF93CDB71B
:10066000DEB766970FB6F894DEBF0FBECDBF7894A5
:1006700084B5826084BD84B5816084BD85B58260A7
:1006800085BD85B5816085BD80916E008160809358
:100690006E001092810080918100826080938100C1
:1006A00080918100816080938100809180008160D1
:1006B000809380008091B10084608093B10080912C
:1006C000B00081608093B00080917A008460809354
:1006D0007A0080917A00826080937A0080917A001B
:1006E000816080937A0080917A00806880937A009C
:1006F0001092C100E0915701F091580112E010836F
:10070000E0915301F09154011082E0915501F09174
:1007100056018FEC808310925F01E0915B01F091B4
:100720005C0186E08083E0915901F0915A0180815B
:1007300080618083E0915901F0915A018081886045
:100740008083E0915901F0915A0180818068808313
:10075000E0915901F0915A0180818F7D808360E0A2
:100760008EE00E94DE0060E08FE00E94DE0060E02C
:1007700080E10E94DE0061E083E00E94DE0062E032
:1007800084E00E94DE0060E081E10E94DE0061E022
:1007900089E00E94DE0061E08AE00E94DE0061E004
:1007A0008BE00E94DE0081EA8093800089E08093E4
:1007B000810083E88093B0001093B100A0E8EA2E96
:1007C000F12CF0928900E0928800F0928B00E09288
:1007D0008A0080E88093B3008FB7F894C0904301FB
:1007E000D0904401E0904501F09046018FBF84E035
:1007F0000E94B5001092F1011092F2019091F00167
:10080000891751F08093F001C092EB01D092EC0176
:10081000E092ED01F092EE018091EB019091EC01FC
:10082000A091ED01B091EE01C81AD90AEA0AFB0ABB
:100830008091E7019091E801A091E901B091EA016E
:100840008C159D05AE05BF05B0F49091EF01809128
:10085000F001981781F08093EF01911103C021E01E
:10086000813009F020E02093F101913009F48111E9
:1008700090E09093F2018091F2018823D1F0609191
:100880003D0181E0682760933D0190E080E00E9497
:10089000F40789E291E00E94390280913D018111C3
:1008A00069C182E291E00E94390285E391E00E94F1
:1008B000390281E10E94B5002091E401211103C0B9
:1008C00091E0813009F090E09093E501213009F446
:1008D000811120E02093E6018093E4019923E1F067
:1008E0000DEC1CEC2CEC3DE300930401109305018E
:1008F000209306013093070110920801109209011C
:1009000010920A0110920B0110920C0110920D012D
:1009100010920E0110920F018EE00E941A01BC018C
:10092000990F880B990B0E94810920E030EC4FE76A
:1009300054E40E94D708362E272E182F9E8B8FE066
:100940000E941A01BC01990F880B990B0E94810922
:1009500020E030EC4FE754E40E94D7082B013C0123
:1009600080E10E941A01BC01990F880B990B0E942B
:10097000810920E030EC4FE754E40E94D7086B0176
:100980007C0100913D010D8B002309F4C5C080E07E
:1009900090E0A0E2B1E48D879E87AF87B88B812C71
:1009A000912CF0E8AF2EFFE3BF2E20E030E0A9014C
:1009B000632D722D812F9E890E94D20887FDBBC0B6
:1009C00020E030E040E85FE3632D722D812F9E89A7
:1009D0000E94310A18160CF0B3C0198200E090E8AA
:1009E0009D83AFE3A987A50194016D857E858F85E1
:1009F00098890E9465082981302F4D8159850E9470
:100A0000360AA50194010E9466084B015C0120E0B2
:100A100030E0A901C301B2010E94D20887FD96C04F
:100A200020E030E040E85FE3C301B2010E94310AF8
:100A3000181634F4412C512C70E8672E7FE3772E82
:100A400020E030E040EF51E4C301B2010E94360AD9
:100A500020E030E040EA51E40E9466086D877E871E
:100A60008F87988B20E030E0A901C701B6010E9472
:100A7000D20887FD6FC020E030E040E85FE3C701A7
:100A8000B6010E94310A181634F4C12CD12C60E84A
:100A9000E62E6FE3F62E20E030E040E450E4C7019C
:100AA000B6010E94360A20E030E040E85FE30E9491
:100AB0006608698B7A8B8B8B9C8B2BE83AE24AEA2F
:100AC0005EE3632D722D812F9E890E94D208181635
:100AD0000CF07EC22BE93AE64AE25FE3632D722D09
:100AE000812F9E890E94D20818160CF046C0ED880E
:100AF0002AE0422E27ED522E23E2622E2CE3722EA4
:100B0000EE2009F44DC08FE6482E82E1582E83E88E
:100B1000682E8AE3782E44C080E090E0A0EAB1E439
:100B20008D879E87AF87B88B812C912CE0EAAE2E03
:100B3000E0E4BE2E3ACF198200E01D82198653CF21
:100B40003982022D1D83BE89B9874DCF412C512C8E
:100B5000320176CFC12CD12C76019DCF1A82198219
:100B600061C12FEF30E03A8329835CC119811E2BCC
:100B70001C9318C286E291E096CEFD889AE0492E39
:100B800097ED592E93EA692E9BE3792EFF2041F0D1
:100B90005FE6452E52E1552E53E0652E5AE3752E41
:100BA0004092000150920101609202017092030193
:100BB000E0900801F090090100910A0110910B01E9
:100BC000E982FA820B831C83C0900401D090050156
:100BD000E0900601F090070100910C0110910D01C9
:100BE00020910E0130910F010D831E832F833887D2
:100BF000A701960169817A818B819C810E94650899
:100C0000A50194010E94360AA30192010E94360AAE
:100C1000A70196010E94660869877A878B879C875F
:100C2000609304017093050180930601909307017E
:100C30002D813E814F8158856D857E858F85988970
:100C40000E946508A70196010E94360A29813A810F
:100C50004B815C810E946508A30192010E94360AC3
:100C600029813A814B815C810E9466084B015C01BD
:100C70008092080190920901A0920A01B0920B01A2
:100C8000A701960169817A818B819C810E94360A35
:100C90006B017C0129893A894B895C896D817E8150
:100CA0008F8198850E94360A9B01AC01C701B6016D
:100CB0000E946508A30192010E94360A2D813E819F
:100CC0004F8158850E94660860930C0170930D0156
:100CD00080930E0190930F01E984FA840B851C85A3
:100CE000202F220F212F221F2F3F61F02A2D220FAC
:100CF0002B2D221F2F3F31F0682F660F692F661FA3
:100D00006F3FE1F40DEC1CEC2CEC3DE3009304018F
:100D100010930501209306013093070110920801FA
:100D20001092090110920A0110920B0110920C010D
:100D300010920D0110920E0110920F0120E030E090
:100D400040EF51E46091040170910501809106012A
:100D5000909107010E94660820E030E04FE753E4DD
:100D60000E94360A20E030E040E752E40E94D708B3
:100D700020E030E0A9010E9466086B017C0120E0C0
:100D800030E0A9010E94D20810E000E087FD11C008
:100D900020E030E04FE753E4C701B6010E94310A7A
:100DA0000FEF10E018162CF0C701B6010E94490998
:100DB0008B0120E030E040EF51E460910801709138
:100DC000090180910A0190910B010E94660820E0C0
:100DD00030E04FE753E40E94360A20E030E040E77D
:100DE00052E40E94D70820E030E0A9010E94660882
:100DF0006B017C0120E030E0A9010E94D20887FD50
:100E0000ADCE20E030E04FE753E4C701B6010E94C9
:100E1000310A18160CF4A5CEC701B6010E94490983
:100E20007A83698320E030E04FE753E460910C015E
:100E300070910D0180910E0190910F010E94360A70
:100E400020E030E048E452E40E94D70820E030E09F
:100E5000A9010E9466086B017C0120E030E0A90135
:100E60000E94D20860E087FD0FC020E030E04FE72D
:100E700053E4C701B6010E94310A6FEF181624F03F
:100E8000C701B6010E9449091093890000938800A8
:100E9000E980FA80F0928B00E0928A006093B300C0
:100EA00020E034E244E759E46091000170910101CF
:100EB00080910201909103010E94360A0E94490923
:100EC0009B01AC012253310941095109AEE3BEEF48
:100ED0000E942F082EED36E240E050E00E9402080A
:100EE000BA01A9014C505E4F6F4F7F4F453F01E063
:100EF00050076105710520F044EF51E060E070E0BB
:100F0000423351056105710520F442E350E060E091
:100F100070E08FB7F894C0904301D0904401E09006
:100F20004501F09046018FBF8091390190913A01BF
:100F3000A0913B01B0913C0197018601081B190B60
:100F40002A0B3B0BD901C801481759076A077B07D1
:100F500008F031C01091380181E018271D831093EB
:100F60003801E1EBF0E08491EDE9F0E004910983D0
:100F7000E9E8F0E014911123B1F081110E948C0096
:100F8000E12FF0E0EE0FFF1FE859FF4FA591B4915C
:100F90008FB7F8941D81EC911111E8CD098100956E
:100FA0000E230C938FBFC0923901D0923A01E09288
:100FB0003B01F0923C0180E090E0892B09F40CCCDD
:100FC0000E949601882309F407CC0E94000004CCFB
:100FD0000D8947E1442E47EB542E41ED642E48E342
:100FE000742E0111DDCD8FCD262FF999FECF1FBABA
:100FF00092BD81BD20BD0FB6F894FA9AF99A0FBE42
:1010000001960895052E97FB1EF400940E9419087E
:1010100057FD07D00E94340807FC03D04EF40C940F
:10102000190850954095309521953F4F4F4F5F4F90
:10103000089590958095709561957F4F8F4F9F4F44
:1010400008950E945608A59F900DB49F900DA49FEF
:10105000800D911D11240895B7FF0C9421080E9462
:101060002108821B930B0895A1E21A2EAA1BBB1B19
:10107000FD010DC0AA1FBB1FEE1FFF1FA217B30764
:10108000E407F50720F0A21BB30BE40BF50B661F7A
:10109000771F881F991F1A9469F76095709580953E
:1010A00090959B01AC01BD01CF010895A29FB001B5
:1010B000B39FC001A39F700D811D1124911DB29F8C
:1010C000700D811D1124911D08955058BB27AA272A
:1010D0000E947D080C94F7090E94E90938F00E94EB
:1010E000F00920F039F49F3F19F426F40C94E60936
:1010F0000EF4E095E7FB0C94E009E92F0E94080A42
:1011000058F3BA17620773078407950720F079F43C
:10111000A6F50C942A0A0EF4E0950B2EBA2FA02DFA
:101120000B01B90190010C01CA01A0011124FF2794
:10113000591B99F0593F50F4503E68F11A16F0408F
:10114000A22F232F342F4427585FF3CF469537958E
:101150002795A795F0405395C9F77EF41F16BA0B53
:10116000620B730B840BBAF09150A1F0FF0FBB1F01
:10117000661F771F881FC2F70EC0BA0F621F731F4A
:10118000841F48F4879577956795B795F7959E3FA7
:1011900008F0B0CF9395880F08F09927EE0F979538
:1011A000879508950E94BC0908F481E008950E9483
:1011B000EB080C94F7090E94F00958F00E94E90925
:1011C00040F029F45F3F29F00C94E00951110C9490
:1011D0002B0A0C94E6090E94080A68F39923B1F3DC
:1011E000552391F3951B550BBB27AA27621773074D
:1011F000840738F09F5F5F4F220F331F441FAA1FE1
:10120000A9F335D00E2E3AF0E0E832D0915050409C
:10121000E695001CCAF72BD0FE2F29D0660F771F4A
:10122000881FBB1F261737074807AB07B0E809F030
:10123000BB0B802DBF01FF2793585F4F3AF09E3FB5
:10124000510578F00C94E0090C942B0A5F3FE4F30D
:10125000983ED4F3869577956795B795F7959F5FF8
:10126000C9F7880F911D9695879597F90895E1E044
:10127000660F771F881FBB1F621773078407BA07A3
:1012800020F0621B730B840BBA0BEE1F88F7E095FE
:1012900008950E9450096894B1110C942B0A089586
:1012A0000E94100A88F09F5798F0B92F9927B751DC
:1012B000B0F0E1F0660F771F881F991F1AF0BA95FA
:1012C000C9F714C0B13091F00E942A0AB1E0089524
:1012D0000C942A0A672F782F8827B85F39F0B93F16
:1012E000CCF3869577956795B395D9F73EF49095AD
:1012F0008095709561957F4F8F4F9F4F0895E8942B
:1013000009C097FB3EF490958095709561957F4F4D
:101310008F4F9F4F9923A9F0F92F96E9BB279395FB
:10132000F695879577956795B795F111F8CFFAF40B
:10133000BB0F11F460FF1BC06F5F7F4F8F4F9F4F3C
:1013400016C0882311F096E911C0772321F09EE89A
:10135000872F762F05C0662371F096E8862F70E000
:1013600060E02AF09A95660F771F881FDAF7880FDA
:101370009695879597F90895990F0008550FAA0B30
:10138000E0E8FEEF16161706E807F907C0F0121698
:101390001306E407F50798F0621B730B840B950B9B
:1013A00039F40A2661F0232B242B252B21F40895F0
:1013B0000A2609F4A140A6958FEF811D811D08958D
:1013C00097F99F6780E870E060E008959FEF80ECF8
:1013D000089500240A94161617061806090608959B
:1013E00000240A9412161306140605060895092E01
:1013F0000394000C11F4882352F0BB0F40F4BF2B70
:1014000011F460FF04C06F5F7F4F8F4F9F4F0895AF
:1014100057FD9058440F551F59F05F3F71F04795A5
:10142000880F97FB991F61F09F3F79F0879508958A
:10143000121613061406551FF2CF4695F1DF08C0A9
:10144000161617061806991FF1CF869571056105C6
:1014500008940895E894BB2766277727CB0197F96E
:1014600008950E94BC0908F48FEF08950E94490A6C
:101470000C94F7090E94E90938F00E94F00920F065
:10148000952311F00C94E0090C94E60911240C94B6
:101490002B0A0E94080A70F3959FC1F3950F50E044
:1014A000551F629FF001729FBB27F00DB11D639F16
:1014B000AA27F00DB11DAA1F649F6627B00DA11DBC
:1014C000661F829F2227B00DA11D621F739FB00D62
:1014D000A11D621F839FA00D611D221F749F3327D2
:1014E000A00D611D231F849F600D211D822F762F6B
:1014F0006A2F11249F5750409AF0F1F088234AF048
:10150000EE0FFF1FBB1F661F771F881F91505040B3
:10151000A9F79E3F510580F00C94E0090C942B0A2A
:101520005F3FE4F3983ED4F3869577956795B7953A
:10153000F795E7959F5FC1F7FE2B880F911D969554
:10154000879597F90895EE0FFF1F0590F491E02D10
:061550000994F894FFCF9E
:101556000AD7233CCDCCCC3D0000000000000000A3
:1015660000000000CC012C01590119028A01680112
:101576007C014F4646004F4E00536C6F77206D6FCF
:0815860064653A20000D0A0023
:00000001FF
